:020000040000FA
:0A00000000000000A4EF00F0BAD0E9
:0800180007D1106E960E076E71
:10002000980E086E6AD8D8B4CA90D8A4CA80FC0FBB
:10003000D8A0CA92D8B0CA82800E076E960E086EFB
:10004000980E0B6E0C6ACAB025D8CAB223D857D8FE
:100050000704CB6E07C009F008C00AF000500D6E0F
:100060000E6E003C0E6A60D80C50102E0AD0BE6E88
:100070000C0EBD6E0BBEBD8A0BBCBD889394CA84AA
:100080001200BB6E0C0EBA6E0BBEBA8A0BBCBA88DD
:100090009492F5D700D8D8900B320832073212006C
:1000A000E836E836FC0B0109C212C009C216C0507E
:1000B000F80B0309C06E320E15D8C282C2B2FED749
:1000C000C4CF14F0C350136E12000A6A096EFF0EFB
:1000D00009260A2200D0D8A01200030E086EE60EF0
:1000E00002D8F5D7086AFE0F076EE86A085AD8A04A
:1000F00012000000070600D0F8D70C6A0B6A100E39
:10010000F36E08340B360C3609500B5C0A500C5851
:1001100005E309500B5E0A500C5AD88007360836A2
:10012000F32EEFD70750120009500D02F3CF0BF05A
:10013000F4CF0CF00A500D02F3500C2609500E02B9
:10014000F3500C260B5012004F0EAF6E240EAC6E07
:10015000900EAB6E00010F0EC16E070EB46EC69A04
:10016000CF0E926EE00E936EC00E946E92849286C5
:10017000020EC06E0D0EC16E010EC26E6CD0F2A4E6
:1001800003D0F294817A11009EAA19D0060EAB1406
:1001900012E1E2CF60F0E1CF5FF0612A10EE83F070
:1001A0006150E126000EE222AECFE7FF60C0E2FF21
:1001B0005FC0E1FF1100AE50AE50AB98AB881100AC
:1001C0006150625C14E0622AEACF08F0E9CF07F0E0
:1001D00000EE83F06250E926000EEA22EF50076E2F
:1001E00008C0EAFF07C0E9FFD880120004D0E86821
:1001F000076ED8A012001200616A626A9D8A9F8A07
:10020000F28EF28C12009D9A00EE83F0010EF46ED5
:10021000F36AF306000EF45AEE6AF450F310F9E1B3
:10022000616A626A9D8A1200F29EE0CF03F8D8CF1D
:1002300004F8E8CF05F8F28E0001A192F29E03C8FF
:10024000E0FF04C8D8FF05C8E8FFF28E10009EA8A2
:10025000FED7AD6E1200939A8A8A0A0E36DF929804
:100260008998929A899A94988B98949A8B9A949058
:100270008B9094968B96010EC26E000E11DF5B6E12
:1002800014C05CF0166A80B4162A166A80B6162A64
:1002900093908A9093928A9293968A9693988A984A
:1002A0000068520E0A6E080E096E010EB6DE006A74
:1002B000520E0A6E080E096E020EAFDE376A366AFB
:1002C000346A00EE68F0180EEE68E82EFDD7356A45
:1002D0004E6A7F0E4F6E4FC065F06690646A636A27
:1002E0004B6A4C6A4D6A3A6A396A3C6A3B6A3E6AB2
:1002F0003D6A426A416A446A436A466A456A486A94
:10030000476A4A6A496A400E806F816B826B74DF6C
:100310007ADFCD6AF294F28A870ED56EB16AA19225
:10032000A082D08EA292B10EB16EEDEC0BF0EFEC8C
:100330000FF0EEEC11F0E7EC15F0030EC26E000EBC
:10034000AFDE5B6E14C05CF0470E5C5C03E346EC12
:100350000BF003D0B7EC0BF04E6A542AE86A54B2A3
:10036000010F55B0010806E15570502A000E5122C8
:100370005222532225DF156EEA0E155C06E3FE0EAF
:10038000155C01E2176ACBEF06F015AE38D0176A9C
:10039000890E155C05E115C017F0186819682DD095
:1003A000990E155C05E115C017F01A681B6825D079
:1003B000A90E155C05E115C017F01C681D681DD05D
:1003C000B90E155C05E115C017F01E681F6815D041
:1003D000C90E155C04E115C017F020680ED0D90EC7
:1003E000155C04E115C017F0216807D0E90E155C13
:1003F00004E115C017F022682368C9EF06F0175210
:1004000004E1CBEF06F0C9EF06F0890E175CD8A423
:100410007CD0182803E115C018F073D015C019F06E
:10042000600E185C05E1349036908998379066D05C
:10043000610E185C05E134903690899A37805ED061
:10044000620E185C08E13490369037B002D089987B
:1004500001D0899A53D0630E185C07E1349234942A
:1004600036923694379E8B9A49D0640E185C06E01B
:10047000650E185C03E0660E185C16E18B868B80B7
:1004800037923794379A3798826B816B0068520E97
:100490000A6E080E096E010E0DEC00F034967768B6
:1004A0007668756874682AD0670E185C18E134980D
:1004B00036988B98379237948B908B963798826BBF
:1004C000816B0068520E0A6E080E096E010E0DEC6B
:1004D00000F0349677687668756874680FD07A0E85
:1004E000185C0CE1006A520E0A6E080E096E020ECC
:1004F0000DEC00F0349A369A4A6A496A1868C9EFD6
:1005000006F0CBEF06F0C9EF06F0990E175CD8A401
:1005100098EF06F01A2804E115C01AF096EF06F0DD
:1005200015C01BF01B52D8A476D0600E1A5C05E1F2
:1005300034903690899837906AD0610E1A5C05E144
:1005400034903690899A378062D0620E1A5C08E146
:100550003490369037B002D0899801D0899A57D01C
:10056000630E1A5C07E13492349436923694379EC7
:100570008B9A4DD0640E1A5C06E0650E1A5C03E09F
:10058000660E1A5C16E18B868B8037943792379A09
:1005900037980068520E0A6E080E096E010E0DECB7
:1005A00000F034967768766875687468826B816B42
:1005B0002ED0670E1A5C19E1349836988B983792D2
:1005C00037948B908B963798379A349677687668FD
:1005D000756874680068520E0A6E080E096E010E86
:1005E0000DEC00F0826B816B12D07A0E1A5C0DE17B
:1005F000006A520E0A6E080E096E020E0DEC00F033
:10060000349A369A4A6A496A02D0CBEF06F0C9EFAB
:1006100006F096EF06F0600E1A5C27E18998899A39
:100620003790348001EE83F0D8901B34E926000E19
:10063000EA22EECF43F0EFCF44F043505024016E56
:1006400044505120026E000E5220036E000E5320C3
:10065000046E04C06BF003C06AF002C069F001C010
:1006600068F08988369094EF06F0610E1A5C27E1F5
:100670008998899A3780348001EE83F0D8901B34B2
:10068000E926000EEA22EECF43F0EFCF44F04350CC
:100690005024016E44505120026E000E5220036E11
:1006A000000E5320046E04C06BF003C06AF002C059
:1006B00069F001C068F0898A369094EF06F0620E06
:1006C0001A5CD8A453D037B003D08998898A02D055
:1006D000899A89883770348001EE83F0D8901B3472
:1006E000E926000EEA22EECF43F0EFCF44F043506C
:1006F0005024016E44505120026E000E5220036EB1
:10070000000E5320046E04C06BF003C06AF002C0F8
:1007100069F001C068F04B5227E0368003EE83F0A9
:10072000D8904B34E926000EEA22EECF01F0EFCF4D
:1007300002F00150435C0250445805E344C03AF0D3
:1007400043C039F011D003EE83F0D8904B34E92642
:10075000000EEA22EECF01F0EFCF02F04350015C31
:10076000396E445002583A6E94EF06F0630E1A5CEC
:10077000D8A457D0348202EE83F0D8901B34E926F7
:10078000000EEA22EECF45F0EFCF46F04550502460
:10079000016E46505120026E000E5220036E000E74
:1007A0005320046E04C06FF003C06EF002C06DF001
:1007B00001C06CF0368204EE83F0D8901B34E92639
:1007C000000EEA22EECF3BF0EFCF3CF04C5221E09E
:1007D000368403EE83F0D8904C34E926000EEA22EA
:1007E000EECF3DF0EFCF3EF03D505024016E3E5035
:1007F0005120026E000E5220036E000E5320046E34
:1008000004C073F003C072F002C071F001C070F058
:1008100006D0379E3694736872687168706894EF7A
:1008200006F0640E1A5CD8A48FD01BC082F08251EF
:10083000815D2EE2812B07EE83F08151EB50006E3B
:10084000520E0A6E080E096E010E0DEC00F0348691
:1008500005EE83F0D8908035E926000EEA22EECF2F
:1008600005F0EFCF06F005505024016E06505120E0
:10087000026E000E5220036E000E5320046E04C060
:1008800077F003C076F002C075F001C074F00ED0AE
:1008900007EE83F01B50EB50006E520E0A6E080EEE
:1008A000096E010E0DEC00F01BC081F0010EC26E4E
:1008B000000E50EC00F05B6E14C05CF0470E5C5C08
:1008C0002BE3000E4EBEFF0E645C07E064504E1832
:1008D000D8B0800A800B0BE003D063504E5C07E277
:1008E0008B908B86379237843788000114D08B80A9
:1008F0008B86379237943798349677687668756820
:1009000074680068520E0A6E080E096E010E0DEC36
:1009100000F0816B826B16D0646A636A8B808B8671
:100920003792379437983496776876687568746824
:10093000826B816B0068520E0A6E080E096E010E02
:100940000DEC00F0379AF0D1650E1A5CD8A489D06E
:100950001BC082F08251815D2EE2812B07EE83F075
:100960008151EB50006E520E0A6E080E096E010E98
:100970000DEC00F0348605EE83F0D8908035E92642
:10098000000EEA22EECF05F0EFCF06F0055050241E
:10099000016E06505120026E000E5220036E000EB2
:1009A0005320046E04C077F003C076F002C075F0E7
:1009B00001C074F010D007EE83F01B50EB50006EB6
:1009C000520E0A6E080E096E010E0DEC00F01BC0EF
:1009D00081F01BC082F0050EC26E470E5E5C2BE3F9
:1009E000000E4FBEFF0E645C07E064504F18D8B095
:1009F000800A800B04E00AD04F50635C07E28B80D2
:100A00008B96379437823788000114D08B808B8681
:100A10003794379237983496776876687568746833
:100A2000816B826B0068520E0A6E080E096E010E11
:100A30000DEC00F014D08B808B863792379437986A
:100A400034967768766875687468826B816B006825
:100A5000520E0A6E080E096E010E0DEC00F0379A68
:100A600063D1660E1A5CD8A4DAD01BC082F0825122
:100A7000815D2EE2812B07EE83F08151EB50006EF9
:100A8000520E0A6E080E096E010E0DEC00F034864F
:100A900005EE83F0D8908035E926000EEA22EECFED
:100AA00005F0EFCF06F005505024016E065051209E
:100AB000026E000E5220036E000E5320046E04C01E
:100AC00077F003C076F002C075F001C074F00ED06C
:100AD00007EE83F01B50EB50006E520E0A6E080EAC
:100AE000096E010E0DEC00F01BC081F0378A6452D4
:100AF000D8A449D04F50635CD8B045D0050EC26E23
:100B0000010E50EC00F05D6E14C05EF0470E5E5CAE
:100B100006E38B808B9637823794378833D08B905F
:100B20008B86379237843788816B348605EE83F065
:100B3000D8908035E926000EEA22EECF05F0EFCFFF
:100B400006F005505024016E06505120026E000E32
:100B50005220036E000E5320046E04C077F003C0D1
:100B600076F002C075F001C074F0812B07EE83F0BF
:100B70008151EB50006E520E0A6E080E096E010E86
:100B80000DEC00F04BD0645204E163504E5CD8B0E1
:100B900045D0010EC26E000E50EC00F05B6E14C02A
:100BA0005CF0470E5C5C000106E38B868B9037841B
:100BB0003792378833D08B968B803794378237883B
:100BC000816B348605EE83F0D8908035E926000EDF
:100BD000EA22EECF05F0EFCF06F005505024016E6B
:100BE00006505120026E000E5220036E000E53205C
:100BF000046E04C077F003C076F002C075F001C047
:100C000074F0812B07EE83F08151EB50006E520E91
:100C10000A6E080E096E010E0DEC00F085D0670E0D
:100C20001A5C37E18B88348801EE83F0D8901B344E
:100C3000E926000EEA22EECF47F0EFCF48F047500A
:100C40005024016E48505120026E000E5220036E57
:100C5000000E5320046E04C07BF003C07AF002C083
:100C600079F001C078F08B808B8637923794379873
:100C7000379A34967768766875687468826B816B8A
:100C80000068520E0A6E080E096E010E0DEC00F09F
:100C90004BD07A0E1A5CD8A445D0D8901B34496E3C
:100CA0004A6A4A367F0E1B5C0AE249C000F0520EC7
:100CB0000A6E080E096E020E0DEC00F00AD04A68AA
:100CC00049680068520E0A6E080E096E020E0DEC9D
:100CD00000F04D5221E0368A06EE83F0D8904D3474
:100CE000E926000EEA22EECF41F0EFCF42F041506C
:100CF0005024016E42505120026E000E5220036EAD
:100D0000000E5320046E04C07FF003C07EF002C0CA
:100D10007DF001C07CF005D0369A7F687E687D68E2
:100D20007C6802D01A6837D01A6833D034D031D0FA
:100D3000A90E175C0BE11C2803E115C01CF004D0C0
:100D400015C01DF094EC09F026D023D0B90E175C25
:100D50000BE11E2803E115C01EF004D015C01FF0E2
:100D60002EEC0AF018D015D0C90E175C08E1202827
:100D700004E115C020F028EC0AF00DD00AD0D90EFD
:100D8000175C07E1212804E115C021F02CEC0AF0E2
:100D900002D05AEC09F0060E5A5CD8B06AD156500F
:100DA000505C575051585850525859505358D8A029
:100DB00051D1598E5A52D8A443D036B008D034906D
:100DC0008998899A6B686A686968686838D034A0BD
:100DD0001BD037B002D0899801D0899A395050245D
:100DE000016E3A505120026E000E5220036E000E2A
:100DF0005320046E04C06BF003C06AF002C069F0B7
:100E000001C068F034901BD037B002D0898A01D07D
:100E10008988377043505024016E44505120026E2F
:100E2000000E5220036E000E5320046E04C06BF0BF
:100E300003C06AF002C069F001C068F0348009D1D3
:100E4000010E5A5C39E136B207D034928B9A6F6842
:100E50006E686D686C682FD034A217D08B9A3B50A7
:100E60005024016E3C505120026E000E5220036E41
:100E7000000E5320046E04C06FF003C06EF002C079
:100E80006DF001C06CF0349216D08B8A455050241E
:100E9000016E46505120026E000E5220036E000E6D
:100EA0005320046E04C06FF003C06EF002C06DF0FA
:100EB00001C06CF03482CDD0020E5A5CD8A43ED072
:100EC00036B406D03494736872687168706835D02F
:100ED000377E3D505024016E3E505120026E000E70
:100EE0005220036E000E5320046E04C073F003C042
:100EF00072F002C071F001C070F0348437BE07D0C8
:100F00008B9A34926F686E686D686C6816D08B8AA5
:100F100045505024016E46505120026E000E522062
:100F2000036E000E5320046E04C06FF003C06EF019
:100F300002C06DF001C06CF034828BD0030E5A5C9D
:100F4000D8A43FD037A837D08251815D2EE2812BC3
:100F500007EE83F08151EB50006E520E0A6E080EC0
:100F6000096E010E0DEC00F0348605EE83F0D8908A
:100F70008035E926000EEA22EECF05F0EFCF06F02D
:100F800005505024016E06505120026E000E522072
:100F9000036E000E5320046E04C077F003C076F099
:100FA00002C075F001C074F005D034967768766899
:100FB0007568746805D03496776876687568746863
:100FC00048D0040E5A5C09E134A806D08B983498B6
:100FD0007B687A68796878683CD0050E5A5C39E19C
:100FE00036BA0ED0349A006A520E0A6E080E096E96
:100FF000020E0DEC00F07F687E687D687C6829D069
:10100000377C37BC09D0006A520E0A6E080E096E92
:10101000020E0DEC00F009D049C000F0520E0A6E2D
:10102000080E096E020E0DEC00F041505024016EC6
:1010300042505120026E000E5220036E000E5320CB
:10104000046E04C07FF003C07EF002C07DF001C0DA
:101050007CF030D953AE0CD0536A526A516A506A50
:10106000346A366A00EE68F0180EEE68E82EFDD796
:1010700006D053AE04D0536A526A516A506A37A8F8
:1010800037D080B433D0675230E137A224D0634ADE
:10109000642A66A014D0000E65BEFF0E645C07E0F3
:1010A00064506518D8B0800A800B07E003D0635005
:1010B000655C03E265C063F0646A00010BD064BE46
:1010C00008D0645203E163507F0803E2646A7F0E34
:1010D000636E000109D037A407D06306000E645A7E
:1010E00064AE02D0646A636A676801D0676A08D038
:1010F00080B405D0675202E16690676801D0676AE4
:1011000037A8D5D037A26BD00D0EC16E050EC26EBA
:10111000010E50EC00F05D6E14C05EF0460EC45C33
:101120000EE28B863792379866A003D065C063F0D5
:10113000646A349677687668756874681AD0000EA9
:101140004FBEFF0E645C07E064504F18D8B0800AB1
:10115000800B0EE003D04F50635C0AE38B8637921E
:10116000379834967768766875687468000101D09E
:101170009ED037AA32D08B908B8637843788010E69
:10118000816F348605EE83F0D8908035E926000E15
:10119000EA22EECF05F0EFCF06F005505024016EA5
:1011A00006505120026E000E5220036E000E532096
:1011B000046E04C077F003C076F002C075F001C081
:1011C00074F007EE83F08151EB50006E520E0A6E00
:1011D000080E096E010E0DEC00F069D068D037A43E
:1011E00066D0010EC26E000E50EC00F05B6E14C0B3
:1011F0005CF0460EC45C0BE28B8037943798646ACF
:10120000636A349677687668756874681AD0000ED9
:101210004EBEFF0E645C07E064504E18D8B0800AE2
:10122000800B04E00DD063504E5C0AE38B80379452
:10123000379834967768766875687468000101D0CD
:1012400036D037AA33D08B808B9637823794378845
:10125000010E816F348605EE83F0D8908035E92643
:10126000000EEA22EECF05F0EFCF06F00550502435
:10127000016E06505120026E000E5220036E000EC9
:101280005320046E04C077F003C076F002C075F0FE
:1012900001C074F007EE83F08151EB50006E520EE6
:1012A0000A6E080E096E010E0DEC00F000D0817080
:1012B000ADEF01F05A68598E166A060E165C33E2DD
:1012C000D8901634E96EEA6AEA36E936EA36680EEC
:1012D000E926000EEA22EFCF01F0ECCF02F0ECCFCE
:1012E00003F0ECCF04F05650015C575002585850B0
:1012F00003585950045815E2D8901634E96EEA6A3A
:10130000EA36E936EA36680EE926000EEA22EFCF21
:1013100056F0ECCF57F0ECCF58F0ECCF59F016C0A8
:101320005AF0162ACAE31200620E1C5C14E11DC0BA
:101330004BF04B520CE003EE83F0D8904B34E9268F
:10134000000EEA22EECF39F0EFCF3AF003D03A6A3E
:10135000396A36907BD0630E1C5C14E11DC04CF0E2
:101360004C520CE003EE83F0D8904C34E926000E8A
:10137000EA22EECF3DF0EFCF3EF003D03E6A3D6A69
:10138000369464D0640E1C5C07E0650E1C5C04E0BF
:10139000660E1C5CD8A444D037A841D01DC082F092
:1013A0008251815D2EE2348605EE83F0D89080353F
:1013B000E926000EEA22EECF05F0EFCF06F0055049
:1013C0005024016E06505120026E000E5220036E12
:1013D000000E5320046E04C077F003C076F002C004
:1013E00075F001C074F0812B07EE83F08151EB5052
:1013F000006E520E0A6E080E096E010E0DEC00F022
:101400000ED01DC081F007EE83F01D50EB50006E32
:10141000520E0A6E080E096E010E0DEC00F016D089
:101420007A0E1C5C13E11DC04DF04D520CE006EE2F
:1014300083F0D8904D34E926000EEA22EECF41F039
:10144000EFCF42F003D0426A416A369A1C6812001C
:101450002068120022681200216812001E0E1E5C15
:1014600035E11F520BE1366A3A6A396A4B6A4C6AB7
:101470003E6A3D6A426A416A4D6A27D01FC04BF0FE
:1014800003EE83F0D8901F34E926000EEA22EECF57
:1014900039F0EFCF3AF01FC04CF003EE83F0D89054
:1014A0001F34E926000EEA22EECF3DF0EFCF3EF0EA
:1014B0001FC04DF006EE83F0D8901F34E926000ED1
:1014C000EA22EECF41F0EFCF42F0ADD0420E1E5CEB
:1014D00007E11F5203E13590A8D801D03580A3D091
:1014E000460E1E5C09E1346A366A8998899A8B989F
:1014F0008B9A8B92CBD897D0470E1E5C06E18B96C9
:101500008B903794379237988ED0480E1E5C1DE131
:1015100065C04FF03496776876687568746807EE32
:1015200083F01F50EB50006E520E0A6E080E096ECB
:10153000010E0DEC00F08B808B9637823794378844
:101540001FC082F01FC081F06ED0490E1E5C1CE1EE
:101550004E6A3496776876687568746807EE83F02B
:101560001F50EB50006E520E0A6E080E096E010EEF
:101570000DEC00F08B908B863792378437881FC034
:1015800082F01FC081F04FD04A0E1E5C0FE11FC0D9
:101590004EF066A005D04F50655C02E265C04FF08A
:1015A0004F504E5C02E34E284F6E3DD04B0E1E5CFA
:1015B0000FE11FC04FF066A005D04F50655C02E2FE
:1015C00065C04FF04F504E5C02E34E284F6E2BD05B
:1015D0004C0E1E5C08E11FC080F0010E805D02E22F
:1015E000010E806F20D07B0E1E5C1DE1346A366ACE
:1015F0008998899A8B988B9A94908B9094968B96D5
:10160000376A826B816B0068520E0A6E080E096E93
:10161000010E0DEC00F0006A520E0A6E080E096E03
:10162000020E0DEC00F01E681200346A366A8998CA
:10163000899A8B988B9A94908B9094968B9600684D
:10164000520E0A6E080E096E010E0DEC00F0006AD3
:10165000520E0A6E080E096E020E0DEC00F0816B40
:10166000826B4E6A66A003D065C04FF002D07F0E39
:101670004F6E376A4B6A4C6A4D6A3A6A396A3E6AFB
:101680003D6A426A416A400E806F1200826B816B34
:101690000068520E0A6E080E096E010E0DEC00F085
:1016A000010EC26E000E50EC00F05B6E14C05CF0D8
:1016B000460EC45C09E28B808B86646A636A4E6A5C
:1016C0003792379437981200050EC26E010E50EC17
:1016D00000F05D6E14C05EF0460EC45C0FE28B90AD
:1016E0008B8637923784378866A004D065C063F054
:1016F000646A03D0646A7F0E636E05D08B908B861C
:10170000379237843788060E816F826FFC0E006E29
:10171000520E0A6E080E096E010E0DEC00F0030E5B
:10172000C26E000E50EC00F05B6E14C05CF0470E11
:10173000C45C09E3010EC26E000E50EC00F05B6E5B
:1017400014C05CF0F4D78B80379237943798646A72
:10175000636A816B826B0068520E0A6E080E096E16
:10176000010E0DEC00F0379A66A001D8120064500B
:101770006310D8A48BDF060E816F826FFC0E006EA3
:10178000520E0A6E080E096E010E0DEC00F08B80F1
:101790008B96379437823788050EC26E010E50EC57
:1017A00000F05D6E14C05EF0470EC45C12E3050EDF
:1017B000C26E010E50EC00F05D6E14C05EF080B49D
:1017C00006D0675203E1634A642A676801D0676AFA
:1017D000EBD763C065F0668059D7030184698369DC
:1017E0005C0E866F7A0E856F590E886F850E876F37
:1017F000580E8A6F140E896F560E8C6FA90E8B6F60
:10180000550E8E6F430E8D6F530E906FE30E8F6FDC
:10181000520E926F890E916F510E946F350E936F29
:101820004F0E966FE60E956F4E0E986F9C0E976F4B
:101830004D0E9A6F580E996F4C0E9C6F190E9B6F40
:101840004A0E9E6FDF0E9D6F490EA06FAA0E9F6F0E
:10185000480EA26F7A0EA16F470EA46F4F0EA36FB2
:10186000460EA66F290EA56F450EA86F080EA76F2E
:10187000430EAA6FEB0EA96F420EAC6FD30EAB6F87
:10188000410EAE6FBF0EAD6F400EB06FB00EAF6FBA
:101890003F0EB26FA50EB16F3E0EB46F9E0EB36FCA
:1018A0003D0EB66F9C0EB56F3C0EB86F9E0EB76FB7
:1018B0003B0EBA6FA40EB96F3A0EBC6FAE0EBB6F83
:1018C000390EBE6FBC0EBD6F380EC06FCE0EBF6F2F
:1018D000370EC26FE30EC16F360EC46FFD0EC36FBD
:1018E000360EC66F1A0EC56F350EC86F3B0EC76F2A
:1018F000340ECA6F5F0EC96F330ECC6F870ECB6F7D
:10190000320ECE6FB20ECD6F310ED06FE10ECF6FB3
:10191000310ED26F140ED16F300ED46F490ED36FCB
:101920002F0ED66F820ED56F2E0ED86FBE0ED76FCC
:101930002D0EDA6FFD0ED96F2D0EDC6F3F0EDB6FB3
:101940002C0EDE6F850EDD6F2B0EE06FCD0EDF6F80
:101950002B0EE26F180EE16F2A0EE46F670EE36F35
:10196000290EE66FB80EE56F290EE86F0C0EE76FD3
:10197000280EEA6F620EE96F270EEC6FBC0EEB6F5C
:10198000270EEE6F180EED6F260EF06F760EEF6FCE
:10199000250EF26FD80EF16F250EF46F3C0EF36F2B
:1019A000240EF66FA20EF56F240EF86F0B0EF76F74
:1019B000230EFA6F760EF96F220EFC6FE40EFB6FAA
:1019C000220EFE6F540EFD6F210E0401006FC60E35
:1019D0000301FF6F210E0401026F3B0E016F200E09
:1019E000046FB20E036F200E066F2B0E056F1F0ED5
:1019F000086FA60E076F1F0E0A6F240E096F1E0ECA
:101A00000C6FA30E0B6F1E0E0E6F250E0D6F1D0EAD
:101A1000106FA90E0F6F1D0E126F2E0E116F1C0E80
:101A2000146FB60E136F1C0E166F3F0E156F1B0E44
:101A3000186FCB0E176F1B0E1A6F580E196F1A0EF8
:101A40001C6FE80E1B6F1A0E1E6F790E1D6F1A0E9B
:101A5000206F0B0E1F6F190E226FA00E216F190E33
:101A6000246F360E236F180E266FCE0E256F180EBC
:101A7000286F680E276F180E2A6F030E296F170E36
:101A80002C6FA00E2B6F170E2E6F3F0E2D6F160EA4
:101A9000306FDF0E2F6F160E326F800E316F160E05
:101AA000346F240E336F150E366FC80E356F150E5A
:101AB000386F6E0E376F150E3A6F160E396F140EA3
:101AC0003C6FBF0E3B6F140E3E6F690E3D6F140EE0
:101AD000406F150E3F6F130E426FC20E416F130E13
:101AE000446F710E436F130E466F210E456F120E39
:101AF000486FD20E476F120E4A6F840E496F120E56
:101B00004C6F380E4B6F110E4E6FED0E4D6F110E68
:101B1000506FA30E4F6F110E526F5A0E516F110E70
:101B2000546F120E536F100E566FCC0E556F100E71
:101B3000586F870E576F100E5A6F420E596F0F0E67
:101B40005C6F5B695E6FBD0E5D6F0F0E606F7C0E2C
:101B50005F6F0F0E626F3D0E616F0E0E646FFE0EB3
:101B6000636F0E0E666FC00E656F0E0E686F830E8C
:101B7000676F0E0E6A6F470E696F0E0E6C6F0C0E5C
:101B80006B6F0D0E6E6FD20E6D6F0D0E706F990E26
:101B90006F6F0D0E726F610E716F0D0E746F2A0EE6
:101BA000736F0C0E766FF40E756F0C0E786FBE0EA1
:101BB000776F0C0E7A6F8A0E796F0C0E7C6F560E53
:101BC0007B6F0C0E7E6F230E7D6F0B0E806FF10E00
:101BD0007F6F0B0E826FC00E816F0601846983696F
:101BE000A20E866FC30E856F9A0E886F460E876FA2
:101BF000960E8A6F320E896F920E8C6F3A0E8B6F33
:101C00008E0E8E6F5D0E8D6F8A0E906F9A0E8F6F97
:101C1000860E926FF00E916F830E946F5F0E936F2E
:101C20007F0E966FE70E956F7C0E986F850E976FFF
:101C3000790E9A6F3B0E996F760E9C6F070E9B6F15
:101C4000720E9E6FE80E9D6F6F0EA06FDF0E9F6F7E
:101C50006C0EA26FEA0EA16F6A0EA46F0A0EA36F3C
:101C6000670EA66F3C0EA56F640EA86F820EA76F5D
:101C7000610EAA6FDA0EA96F5F0EAC6F440EAB6FE8
:101C80005C0EAE6FBF0EAD6F5A0EB06F4C0EAF6FE5
:101C9000570EB26FE90EB16F550EB46F960EB36F5B
:101CA000530EB66FB56F510EB86F200EB76F4E0E54
:101CB000BA6FFB0EB96F4C0EBC6FE50EBB6F4A0ED0
:101CC000BE6FDC0EBD6F480EC06FE20EBF6F460EDA
:101CD000C26FF50EC16F450EC46F150EC36F430E74
:101CE000C66F420EC56F410EC86F7B0EC76F3F0EA9
:101CF000CA6FC00EC96F3E0ECC6F100ECB6F3C0E7C
:101D0000CE6F6D0ECD6F3A0ED06FD40ECF6F390EF1
:101D1000D26F460ED16F370ED46FC20ED36F360E10
:101D2000D66F490ED56F340ED86FDA0ED76F330EDB
:101D3000DA6F740ED96F320EDC6F180EDB6F300E57
:101D4000DE6FC50EDD6F2F0EE06F7B0EDF6F2E0E88
:101D5000E26F3A0EE16F2D0EE46F020EE36F2B0E71
:101D6000E66FD10EE56F2A0EE86FA90EE76F290E18
:101D7000EA6F880EE96F280EEC6F6F0EEB6F270E7F
:101D8000EE6F5E0EED6F260EF06F530EEF6F250EA9
:101D9000F26F500EF16F240EF46F540EF36F230E9A
:101DA000F66F5E0EF56F220EF86F6F0EF76F210E55
:101DB000FA6F860EF96F200EFC6FA30EFB6F1F0EDD
:101DC000FE6FC60EFD6F1E0E0701006FEF0E0601BF
:101DD000FF6F1E0E0701026F016F1D0E046F520E82
:101DE000036F1C0E066F8C0E056F1B0E086FCB0E5B
:101DF000076F1B0E0A6F0F0E096F1A0E0C6F580E2D
:101E00000B6F190E0E6FA50E0D6F180E106FF80EDA
:101E10000F6F180E126F4F0E116F170E146FAB0E5F
:101E2000136F170E166F0A0E156F160E186F6F0EC2
:101E3000176F150E1A6FD70E196F150E1C6F430E04
:101E40001B6F140E1E6FB30E1D6F140E206F270E26
:101E50001F6F130E226F9F0E216F130E246F1A0E29
:101E6000236F120E266F990E256F120E286F1B0E10
:101E7000276F110E2A6FA10E296F110E2C6F290EDC
:101E80002B6F100E2E6FB50E2D6F100E306F440E8F
:101E90002F6F0F0E326FD60E316F0F0E346F6B0E29
:101EA000336F0F0E366F030E356F0E0E386F9D0EAB
:101EB000376F0E0E3A6F3A0E396F0D0E3C6FDA0E19
:101EC0003B6F0D0E3E6F7C0E3D6F0D0E406F210E71
:101ED0003F6F0C0E426FC80E416F0C0E446F720EB6
:101EE000436F0C0E466F1E0E456F0B0E486FCC0EE7
:101EF000476F0B0E4A6F7C0E496F0B0E4C6F2E0E08
:101F00004B6F0A0E4E6FE30E4D6F0A0E506F990E17
:101F10004F6F0A0E526F510E516F0A0E546F0B0E17
:101F2000536F090E566FC80E556F090E586F850E08
:101F3000576F090E5A6F450E596F090E5C6F060EEA
:101F40005B6F080E5E6FC90E5D6F080E606F8E0EC0
:101F50005F6F080E626F540E616F080E646F1C0E87
:101F6000636F070E666FE50E656F070E686FAF0E45
:101F7000676F070E6A6F7B0E696F070E6C6F490EF5
:101F80006B6F070E6E6F170E6D6F060E706FE70E9C
:101F90006F6F060E726FB90E716F060E746F8B0E37
:101FA000736F060E766F5F0E756F060E786F340EC8
:101FB000776F060E7A6F0A0E796F050E7C6FE10E51
:101FC0007B6F050E7E6FB90E7D6F050E806F930ED1
:101FD0007F6F050E826F6D0E816F00011200040E7F
:101FE0000101866F880E856F040E886FA60E876FBD
:101FF000040E8A6FB60E896F040E8C6FC60E8B6F3F
:10200000040E8E6FD60E8D6F040E906FE60E8F6FDE
:10201000040E926FF60E916F050E946F070E936F7C
:10202000050E966F170E956F050E986F280E976F19
:10203000050E9A6F390E996F050E9C6F4B0E9B6FB4
:10204000050E9E6F5D0E9D6F050EA06F6E0E9F6F4D
:10205000050EA26F800EA16F050EA46F930EA36FE5
:10206000050EA66FA50EA56F050EA86FB80EA76F7B
:10207000050EAA6FCB0EA96F050EAC6FDF0EAB6F0E
:10208000050EAE6FF20EAD6F060EB06FAF6FB26F92
:102090001A0EB16F060EB46F2E0EB36F060EB66F2A
:1020A000430EB56F060EB86F580EB76F060EBA6FB7
:1020B0006D0EB96F060EBC6F830EBB6F060EBE6F42
:1020C000980EBD6F060EC06FAE0EBF6F060EC26FCC
:1020D000C40EC16F060EC46FDB0EC36F060EC66F53
:1020E000F20EC56F070EC86F090EC76F070ECA6FD5
:1020F000210EC96F070ECC6F380ECB6F070ECE6F57
:10210000500ECD6F070ED06F690ECF6F070ED26FD6
:10211000810ED16F070ED46F9A0ED36F070ED66F54
:10212000B40ED56F070ED86FCD0ED76F070EDA6FCE
:10213000E70ED96F080EDC6F020EDB6F080EDE6F44
:102140001D0EDD6F080EE06F380EDF6F080EE26FB8
:10215000530EE16F080EE46F6F0EE36F080EE66F2B
:102160008B0EE56F080EE86FA70EE76F080EEA6F9B
:10217000C40EE96F080EEC6FE10EEB6F080EEE6F08
:10218000ED69090EF06F1D0EEF6F090EF26F3B0E39
:10219000F16F090EF46F5A0EF36F090EF66F790E98
:1021A000F56F090EF86F990EF76F090EFA6FB90EF9
:1021B000F96F090EFC6FD90EFB6F090EFE6FFA0E58
:1021C000FD6F0A0E0201006F1B0E0101FF6F0A0E68
:1021D0000201026F3D0E016F0A0E046F5F0E036F66
:1021E0000A0E066F820E056F0A0E086FA50E076FA6
:1021F0000A0E0A6FC80E096F0A0E0C6FEC0E0B6FF9
:102200000B0E0E6F110E0D6F0B0E106F360E0F6F43
:102210000B0E126F5B0E116F0B0E146F810E136F8E
:102220000B0E166FA70E156F0B0E186FCE0E176FD5
:102230000B0E1A6FF50E196F0C0E1C6F1D0E1B6F17
:102240000C0E1E6F460E1D6F0C0E206F6F0E1F6F53
:102250000C0E226F980E216F0C0E246FC20E236F8E
:102260000C0E266FED0E256F0D0E286F180E276FC2
:102270000D0E2A6F430E296F0D0E2C6F700E2B6FF3
:102280000D0E2E6F9C0E2D6F0D0E306FCA0E2F6F20
:102290000D0E326FF80E316F0E0E346F260E336F47
:1022A0000E0E366F550E356F0E0E386F850E376F6A
:1022B0000E0E3A6FB60E396F0E0E3C6FE70E3B6F87
:1022C0000F0E3E6F180E3D6F0F0E406F4B0E3F6F9F
:1022D0000F0E426F7E0E416F0F0E446FB10E436FB3
:1022E0000F0E466FE60E456F100E486F1B0E476FC0
:1022F000100E4A6F500E496F100E4C6F870E4B6FC9
:10230000100E4E6FBE0E4D6F100E506FF60E4F6FCB
:10231000110E526F2E0E516F110E546F680E536FC7
:10232000110E566FA20E556F110E586FDC0E576FBF
:10233000120E5A6F180E596F120E5C6F540E5B6FAF
:10234000120E5E6F910E5D6F120E606FCF0E5F6F9B
:10235000130E626F0E0E616F130E646F4D0E636F7E
:10236000130E666F8E0E656F130E686FCF0E676F5C
:10237000140E6A6F110E696F140E6C6F540E6B6F32
:10238000140E6E6F980E6D6F140E706FDC0E6F6F03
:10239000150E726F220E716F150E746F680E736FCB
:1023A000150E766FB00E756F150E786FF80E776F8D
:1023B000160E7A6F410E796F160E7C6F8C0E7B6F46
:1023C000160E7E6FD70E7D6F170E806F230E7F6FF8
:1023D000170E826F700E816F00011200160E04013D
:1023E000866F500E856F160E886F230E876F150E41
:1023F0008A6FF60E896F150E8C6FC90E8B6F150ED6
:102400008E6F9C0E8D6F150E906F6F0E8F6F150E69
:10241000926F420E916F150E946F936F140E966F1C
:10242000E80E956F140E986FBB0E976F140E9A6F8F
:102430008E0E996F140E9C6F610E9B6F140E9E6F23
:10244000340E9D6F140EA06F070E9F6F130EA26FB8
:10245000DA0EA16F130EA46FAD0EA36F130EA66F4D
:10246000800EA56F130EA86F530EA76F130EAA6FE1
:10247000260EA96F120EAC6FF90EAB6F120EAE6F77
:10248000CC0EAD6F120EB06F9F0EAF6F120EB26F0B
:10249000720EB16F120EB46F450EB36F120EB66F9F
:1024A000180EB56F110EB86FEB0EB76F110EBA6F35
:1024B000BE0EB96F110EBC6F910EBB6F110EBE6FC9
:1024C000640EBD6F110EC06F370EBF6F110EC26F5D
:1024D0000A0EC16F100EC46FDD0EC36F100EC66FF3
:1024E000B00EC56F100EC86F830EC76F100ECA6F87
:1024F000560EC96F100ECC6F290ECB6F0F0ECE6F1C
:10250000FC0ECD6F0F0ED06FCF0ECF6F0F0ED26FB0
:10251000A20ED16F0F0ED46F750ED36F0F0ED66F44
:10252000480ED56F0F0ED86F1B0ED76F0E0EDA6FD9
:10253000EE0ED96F0E0EDC6FC10EDB6F0E0EDE6F6E
:10254000940EDD6F0E0EE06F670EDF6F0E0EE26F02
:102550003A0EE16F0E0EE46F0D0EE36FE66FE00EC4
:10256000E56F0D0EE86FB30EE76F0D0EEA6F860E86
:10257000E96F0D0EEC6F590EEB6F0D0EEE6F2C0E1A
:10258000ED6F0C0EF06FEF69F26FD20EF16F0C0E63
:10259000F46FA50EF36F0C0EF66F780EF56F0C0E40
:1025A000F86F4B0EF76F0C0EFA6F1E0EF96F0B0ED5
:1025B000FC6FF10EFB6F0B0EFE6FC40EFD6F0B0E6A
:1025C0000501006F970E0401FF6F0B0E0501026FEE
:1025D0006A0E016F0B0E046F3D0E036F0B0E066F3C
:1025E000100E056F0A0E086FE30E076F0A0E0A6FD2
:1025F000B60E096F0A0E0C6F890E0B6F0A0E0E6F66
:102600005C0E0D6F0A0E106F2F0E0F6F0A0E126FF9
:10261000020E116F090E146FD50E136F090E166F8F
:10262000A80E156F090E186F7B0E176F090E1A6F23
:102630004E0E196F090E1C6F210E1B6F080E1E6FB8
:10264000F40E1D6F080E206FC70E1F6F080E226F4D
:102650009A0E216F080E246F6D0E236F080E266FE1
:10266000400E256F080E286F130E276F070E2A6F76
:10267000E60E296F070E2C6FB90E2B6F070E2E6F0B
:102680008C0E2D6F070E306F5F0E2F6F070E326F9F
:10269000320E316F070E346F050E336F060E366F34
:1026A000D80E356F060E386FAB0E376F060E3A6FC9
:1026B0007E0E396F060E3C6F510E3B6F060E3E6F5D
:1026C000240E3D6F050E406FF70E3F6F050E426FF3
:1026D000CA0E416F050E446F9D0E436F050E466F87
:1026E000700E456F050E486F430E476F050E4A6F1B
:1026F000160E496F040E4C6FE90E4B6F040E4E6FB1
:10270000BC0E4D6F040E506F8F0E4F6F040E526F44
:10271000620E516F040E546F350E536F040E566FD8
:10272000080E556F030E586FDB0E576F030E5A6F6E
:10273000AE0E596F030E5C6F810E5B6F030E5E6F02
:10274000540E5D6F030E606F270E5F6F020E626F97
:10275000FA0E616F020E646FCD0E636F020E666F2C
:10276000A00E656F020E686F730E676F020E6A6FC0
:10277000460E696F020E6C6F190E6B6F010E6E6F55
:10278000EC0E6D6F010E706FBF0E6F6F010E726FEA
:10279000920E716F010E746F650E736F010E766F7E
:1027A000380E756F010E786F0B0E776F7A6BDE0E39
:1027B000796F7C6BB10E7B6F7E6B840E7D6F806B4F
:1027C000570E7F6F826B2A0E816F050E0201866F96
:1027D000940E856F050E886FC10E876F050E8A6F88
:1027E000EE0E896F060E8C6F1B0E8B6F060E8E6FB2
:1027F000480E8D6F060E906F750E8F6F060E926FDE
:10280000A20E916F060E946FCF0E936F060E966F09
:10281000FC0E956F070E986F290E976F070E9A6F33
:10282000560E996F070E9C6F830E9B6F070E9E6F5F
:10283000B00E9D6F070EA06FDD0E9F6F080EA26F8A
:102840000A0EA16F080EA46F370EA36F080EA66FB5
:10285000640EA56F080EA86F910EA76F080EAA6FE1
:10286000BE0EA96F080EAC6FEB0EAB6F090EAE6F0C
:10287000180EAD6F090EB06F450EAF6F090EB26F37
:10288000720EB16F090EB46F9F0EB36F090EB66F63
:10289000CC0EB56F090EB86FF90EB76F0A0EBA6F8E
:1028A000260EB96F0A0EBC6F530EBB6F0A0EBE6FB9
:1028B000800EBD6F0A0EC06FAD0EBF6F0A0EC26FE5
:1028C000DA0EC16F0B0EC46F070EC36F0B0EC66F0F
:1028D000340EC56F0B0EC86F610EC76F0B0ECA6F3B
:1028E0008E0EC96F0B0ECC6FBB0ECB6F0B0ECE6F67
:1028F000E80ECD6F0C0ED06F150ECF6F0C0ED26F91
:10290000420ED16F0C0ED46F6F0ED36F0C0ED66FBC
:102910009C0ED56F0C0ED86FC90ED76F0C0EDA6FE8
:10292000F60ED96F0D0EDC6F230EDB6F0D0EDE6F12
:10293000500EDD6F0D0EE06F7D0EDF6F0D0EE26F3E
:10294000AA0EE16F0D0EE46FD70EE36F0E0EE66F69
:10295000040EE56F0E0EE86F310EE76F0E0EEA6F94
:102960005E0EE96F0E0EEC6F8B0EEB6F0E0EEE6FC0
:10297000B80EED6F0E0EF06FE50EEF6F0F0EF26FEB
:10298000120EF16F0F0EF46F3F0EF36F0F0EF66F16
:102990006C0EF56F0F0EF86F990EF76F0F0EFA6F42
:1029A000C60EF96F0F0EFC6FF30EFB6F100EFE6F6D
:1029B000200EFD6F100E0301006F4D0E0201FF6F20
:1029C000100E0301026F7A0E016F100E046FA70E36
:1029D000036F100E066FD40E056F110E086F010EF7
:1029E000076F110E0A6F2E0E096F110E0C6F5B0E22
:1029F0000B6F110E0E6F880E0D6F110E106FB50E4E
:102A00000F6F110E126FE20E116F120E146F0F0E78
:102A1000136F120E166F3C0E156F120E186F690EA3
:102A2000176F120E1A6F960E196F120E1C6FC30ECF
:102A30001B6F120E1E6FF00E1D6F130E206F1D0EFA
:102A40001F6F130E226F4A0E216F130E246F770E25
:102A5000236F130E266FA40E256F130E286FD10E51
:102A6000276F130E2A6FFE0E296F140E2C6F2B0E7C
:102A70002B6F140E2E6F580E2D6F140E306F850EA7
:102A80002F6F140E326FB20E316F140E346FDF0ED3
:102A9000336F150E366F0C0E356F150E386F390EFD
:102AA000376F150E3A6F660E396F150E3C6F930E29
:102AB0003B6F150E3E6FC00E3D6F150E406FED0E55
:102AC0003F6F160E426F1A0E416F160E446F470E7F
:102AD000436F160E466F740E456F160E486FA10EAB
:102AE000476F160E4A6FCE0E496F160E4C6FFB0ED7
:102AF0004B6F170E4E6F280E4D6F170E506F550E01
:102B00004F6F170E526F820E516F170E546FAF0E2C
:102B1000536F170E566FDC0E556F180E586F090E57
:102B2000576F180E5A6F360E596F180E5C6F630E82
:102B30005B6F180E5E6F900E5D6F180E606FBD0EAE
:102B40005F6F180E626FEA0E616F190E646F170ED9
:102B5000636F190E666F440E656F190E686F710E04
:102B6000676F190E6A6F9E0E696F190E6C6FCB0E30
:102B70006B6F190E6E6FF80E6D6F1A0E706F250E5B
:102B80006F6F1A0E726F520E716F1A0E746F7F0E86
:102B9000736F1A0E766FAC0E756F1A0E786FD90EB2
:102BA000776F1B0E7A6F060E796F1B0E7C6F330EDC
:102BB0007B6F1B0E7E6F600E7D6F1B0E806F8D0E08
:102BC0007F6F1B0E826FBA0E816F0001120007012A
:102BD0008369FD0E846FFC0E856FFB0E866FFA0E07
:102BE000876FF90E886FF80E896F8A6FF70E8B6FFB
:102BF0008C6FF60E8D6F8E6FF50E8F6F906FF40EDB
:102C0000916F926FF30E936F946FF20E956F966FB4
:102C1000F10E976F986FF00E996F9A6FEF0E9B6F92
:102C20009C6FEE0E9D6F9E6FED0E9F6FA06FEC0E72
:102C3000A16FA26FEB0EA36FA46FEA0EA56FA66F34
:102C4000E90EA76FA86FE80EA96FAA6FE70EAB6F2A
:102C5000AC6FE60EAD6FAE6FE50EAF6FB06FE40E0A
:102C6000B16FB26FE30EB36FB46FE20EB56FB66FB4
:102C7000E10EB76FB86FE00EB96FBA6FDF0EBB6FC2
:102C8000BC6FDE0EBD6FBE6FDD0EBF6FC06FDC0EA2
:102C9000C16FC26FDB0EC36FC46FDA0EC56FC66F34
:102CA000D90EC76FC86FD80EC96FCA6FD70ECB6F5A
:102CB000CC6FCD6FD60ECE6FCF6FD50ED06FD16FDC
:102CC000D40ED26FD36FD30ED46FD56FD20ED66F12
:102CD000D76FD10ED86FD96FD00EDA6FDB6FCF0EF2
:102CE000DC6FDD6FCE0EDE6FDF6FCD0EE06FE16F5C
:102CF000CC0EE26FE36FCB0EE46FE56FCA0EE66FAA
:102D0000E76FC90EE86FE96FC80EEA6FEB6FC70E89
:102D1000EC6FED6FC60EEE6FEF6FC50EF06FF16FDB
:102D2000C40EF26FF36FC30EF46FF56FC20EF66F41
:102D3000F76FC10EF86FF96FC00EFA6FFB6FBF0E21
:102D4000FC6FFD6FBE0EFE6FFF6FBD0E0801006FC2
:102D5000016FBC0E026F150E0501846F7C0E836F30
:102D6000160E866F610E856F150E886FAA0E876F1F
:102D7000140E8A6FF80E896F140E8C6F4D0E8B6FC8
:102D8000130E8E6FA70E8D6F130E906F060E8F6F42
:102D9000120E926F6A0E916F110E946FD30E936F95
:102DA000110E966F420E956F100E986FB40E976FBE
:102DB000100E9A6F2C0E996F0F0E9C6FA70E9B6FC3
:102DC0000F0E9E6F270E9D6F0E0EA06FAB0E9F6FA6
:102DD0000E0EA26F330EA16F0D0EA46FBF0EA36F68
:102DE0000D0EA66F4E0EA56F0C0EA86FE10EA76F0D
:102DF0000C0EAA6F780EA96F0C0EAC6F120EAB6F93
:102E00000B0EAE6FAF0EAD6F0B0EB06F500EAF6FFF
:102E10000A0EB26FF30EB16F0A0EB46F990EB36F54
:102E20000A0EB66F430EB56F090EB86FEF0EB76F8F
:102E3000090EBA6F9D0EB96F090EBC6F4F0EBB6FB6
:102E4000090EBE6F030EBD6F080EC06FB90EBF6FC7
:102E5000080EC26F710EC16F080EC46F2C0EC36FC7
:102E6000070EC66FE90EC56F070EC86FA90EC76FB4
:102E7000070ECA6F6A0EC96F070ECC6F2D0ECB6F8F
:102E8000060ECE6FF30ECD6F060ED06FBA0ECF6F5B
:102E9000060ED26F830ED16F060ED46F4D0ED36F18
:102EA000060ED66F1A0ED56F050ED86FE80ED76FC7
:102EB000050EDA6FB80ED96F050EDC6F890EDB6F69
:102EC000050EDE6F5B0EDD6F050EE06F300EDF6FFF
:102ED000050EE26FE16F040EE46FDC0EE36F040E8B
:102EE000E66FB40EE56F040EE86F8E0EE76F040E0A
:102EF000EA6F690EE96F040EEC6F440EEB6F040E7F
:102F0000EE6F220EED6F040EF06FEF6B030EF26F9B
:102F1000DF0EF16F030EF46FBF0EF36F030EF66F4B
:102F2000A10EF56F030EF86F830EF76F030EFA6FA5
:102F3000660EF96F030EFC6F4A0EFB6F030EFE6FF9
:102F40002F0EFD6F030E0601006F150E0501FF6FBA
:102F5000020E0601026FFC0E016F020E046FE40EFA
:102F6000036F020E066FCC0E056F020E086FB50ED2
:102F7000076F020E0A6F9F0E096F020E0C6F8A0E0A
:102F80000B6F020E0E6F750E0D6F020E106F610E3D
:102F90000F6F020E126F4D0E116F020E146F3A0E6C
:102FA000136F020E166F280E156F020E186F170E94
:102FB000176F020E1A6F050E196F010E1C6FF50EBA
:102FC0001B6F010E1E6FE50E1D6F010E206FD50EDB
:102FD0001F6F010E226FC60E216F010E246FB80EF7
:102FE000236F010E266FAA0E256F010E286F9C0E0F
:102FF000276F010E2A6F8F0E296F010E2C6F820E24
:103000002B6F010E2E6F760E2D6F010E306F6A0E34
:103010002F6F010E326F5E0E316F010E346F530E43
:10302000336F010E366F480E356F010E386F3E0E4E
:10303000376F010E3A6F340E396F010E3C6F2A0E56
:103040003B6F010E3E6F200E3D6F010E406F170E5D
:103050003F6F010E426F0E0E416F010E446F060E60
:10306000436F466BFD0E456F486BF50E476F4A6B1D
:10307000ED0E496F4C6BE60E4B6F4E6BDE0E4D6FD7
:10308000506BD70E4F6F526BD00E516F546BCA0EF0
:10309000536F566BC30E556F586BBD0E576F5A6BFF
:1030A000B70E596F5C6BB10E5B6F5E6BAB0E5D6FF5
:1030B000606BA60E5F6F626BA10E616F646B9C0EFE
:1030C000636F666B970E656F686B920E676F6A6BC6
:1030D0008D0E696F6C6B890E6B6F6E6B840E6D6FEE
:1030E000706B800E6F6F726B7C0E716F746B780EED
:1030F000736F766B740E756F786B700E776F7A6B7B
:103100006D0E796F7C6B690E7B6F7E6B660E7D6FCB
:10311000806B630E7F6F826B600E816F0001120007
:02312000FFD7D7
:020000040030CA
:0300010006160ED2
:020005008580F4
:060008000FC00FE00F40E5
:00000001FF
